:100000000C9468000C9490000C9490000C94900058
:100010000C9490000C9490000C9490000C94900020
:100020000C9490000C9490000C9490000C94900010
:100030000C9490000C9490000C9490000C94900000
:100040000C945C070C9490000C9490000C9490001D
:100050000C9490000C9490000C9490000C949000E0
:100060000C948A040C949000000000090003020024
:10007000000405080000000000000000000000016E
:10008000020408102040800102040810200102042C
:100090000810204080400404040404040404020204
:1000A000020202020303030303030202030000002F
:1000B0000023002600290000000000250028002B56
:1000C0000000000000240027002A0000BF021604E0
:1000D00011241FBECFEFD8E0DEBFCDBF11E0A0E0FE
:1000E000B1E0ECE4F5E102C005900D92A832B10751
:1000F000D9F723E0A8E2B1E001C01D92A53BB20709
:10010000E1F710E0C8E6D0E004C02197FE010E94AC
:100110009E0AC636D107C9F70E945D090C94A40A4D
:100120000C940000CF93DF9369E089EE92E00E9487
:10013000090461E085E00E94C90861E089E00E944D
:10014000C90861E08AE00E94C908C3E0D1E062E02A
:1001500089910E94C90881E0C930D807C1F770E0D1
:1001600060E085E00E94430870E060E089E00E9462
:10017000430870E060E08AE00E9443081092D302D6
:100180001092D4021092D5021092D6021092D70289
:100190001092D8021092E2021092E3021092E4024E
:1001A0001092E5021092E6021092E7021092E80225
:1001B000DF91CF9108950F931F93CF93DF938B011E
:1001C000EA01BC0185E00E944308B80189E00E9471
:1001D0004308BE018AE0DF91CF911F910F910C94EB
:1001E000430850E040E070E060E090E080E00C9474
:1001F000DB008230A9F028F4882341F0813041F0FF
:1002000008958330A1F08430B9F008950C94F10082
:1002100050E040E070E060E08FEF90E00C94DB0095
:1002200050E040E06FEF70E090E080E0F7CF4FEFFC
:1002300050E070E060E0F8CF4FE750E06FE770E02B
:100240008FE790E0EBCFFF920F931F93CF93DF9355
:100250001092020108E211E0D0E0C0E0FC2E6EE155
:10026000C8010E94CD066093D9027093DA02809390
:10027000DB029093DC0260327340810591050CF43F
:100280007CC0E091E102EE2351F0F0E0EF51FD4F30
:100290002081CE0101962817190609F46EC083E06B
:1002A0000E94F9008091E102E82FF0E0EE51FD4F4D
:1002B000F394F0828F5F8093E1020E94A60760931F
:1002C000DD027093DE028093DF029093E0021092D1
:1002D000010168E572E080E090E00E94D7070E948B
:1002E000F1008091E102873001F590910201A2EEC8
:1002F000B2E0EFE0F1E080E03D912191321709F4A6
:1003000044C01092020180910201813009F047C07F
:1003100082E00E94F90060E777E180E090E00E94CF
:10032000D707109202010E94F1008091E10287300C
:1003300009F03FC08091E102873059F084E00E94CB
:10034000F90068E572E080E090E00E94D7070E9423
:10035000F1001092E2021092E3021092E402109275
:10036000E5021092E6021092E7021092E80281E0A4
:10037000809301011092E10234C02196025E1F4F6A
:10038000C730D10509F06ACFACCF863009F491E0CF
:100390008F5F873009F0B0CF90930201B4CF81E036
:1003A0000E94F90068EB7BE080E090E00E94D707B4
:1003B000BACF0E94A6070091DD021091DE022091C3
:1003C000DF023091E002601B710B820B930B6031F6
:1003D00077428105910528F080910101882309F475
:1003E000A9CFDF91CF911F910F91FF9008950F93A7
:1003F0001F93CF931092CD0203E011E0C0E0F8010B
:1004000081918F010E9433098093CC02CF5F8111CB
:1004100078C0E091D202EE2359F0F0E0EE52FD4FA9
:100420002081C801835091402817190609F469C03A
:1004300083E00E94F90068E572E080E090E00E94AD
:10044000D7070E94F1008091D202E82FF0E0ED5230
:10045000FD4FC0838F5F8093D2020E94A6076093F6
:10046000CE027093CF028093D0029093D10210926B
:1004700000018091D2028630F9F49091CD02A3ED73
:10048000B2E0E9E0F1E080E03D9121913217E9F13D
:100490001092CD028091CD02813009F040C082E0FF
:1004A0000E94F90060E777E180E090E00E94D707C2
:1004B0001092CD020E94F1008091D2028630C9F5DF
:1004C0008091D202863059F084E00E94F90068E5FC
:1004D00072E080E090E00E94D7070E94F100109245
:1004E000D3021092D4021092D5021092D60210922A
:1004F000D7021092D80281E0809300011092D202BC
:1005000030C0C63009F07BCFB4CF853009F491E01C
:100510008F5F863009F0B8CF9093CD02BBCF81E0DA
:100520000E94F90068EB7BE080E090E00E94D70732
:10053000C1CF0E94A6070091CE021091CF02209158
:10054000D0023091D102601B710B820B930B603192
:1005500077428105910528F080910001882309F4F4
:10056000AFCFCF911F910F91089569E273E089EEAB
:1005700092E00E9411040E9423010C94F70140E1D3
:100580006FE08EEA92E00E94AA0541E16FE080E907
:1005900092E00E94AA0540E06FE082E792E00E94AC
:1005A000AA0541E06FE084E592E00E94AA0542E0DE
:1005B0006FE086E392E00E94AA0543E06FE088E1E5
:1005C00092E00E94AA0544E06FE08AEF91E00E9469
:1005D000AA058EE1EEEAF2E0A8E2B1E001900D9208
:1005E0008A95E1F78EE1E0E9F2E0A6E4B1E001905E
:1005F0000D928A95E1F78EE1E2E7F2E0A4E6B1E040
:1006000001900D928A95E1F78EE1E4E5F2E0A2E82F
:10061000B1E001900D928A95E1F78EE1E6E3F2E018
:10062000A0EAB1E001900D928A95E1F78EE1E8E150
:10063000F2E0AEEBB1E001900D928A95E1F78EE128
:10064000EAEFF1E0ACEDB1E001900D928A95E1F7AF
:1006500008958091020161E0813031F08091CD02F6
:1006600062E0813009F060E089EE92E00C949B0337
:1006700090E080E0089580911C0390911D03891BF8
:10068000990B089590911D0380911C032FEF3FEF6C
:10069000981748F4E92FF0E0E25EFC4F208130E04B
:1006A0009F5F90931D03C9010895E0911D03809100
:1006B0001C03E81730F4F0E0E25EFC4F808190E02C
:1006C00008958FEF9FEF08950895CF93DF93EC0186
:1006D000E091F502F091F6023097F1F090911D0350
:1006E00080911C039817C0F090E0292F30E0261766
:1006F000370754F4DE01A20FB31F4C91225E3C4F2A
:10070000D9014C939F5FF1CF10921D0360931C039E
:10071000CB01DF91CF910994DF91CF910895E091C2
:10072000F702F091F802309729F01092FB02109234
:10073000FA0209940895CF93DF931F92CDB7DEB7E5
:1007400069832091F9022223F9F02091FA022032E4
:1007500058F021E030E0FC013383228390E080E018
:100760000F90DF91CF9108958091FB02E82FF0E088
:10077000E450FD4F998190838F5F8093FB028093BB
:10078000FA0281E090E0ECCF61E0CE0101960E9498
:100790004904F7CFCF92DF92EF92FF920F931F930E
:1007A000CF93DF937C01CB018A012091F9022223B0
:1007B00089F0EB016B01C40ED51ECC15DD0569F087
:1007C0006991D701ED91FC910190F081E02DC70175
:1007D0000995F3CF642F0E944904C801DF91CF919E
:1007E0001F910F91FF90EF90DF90CF90089510929E
:1007F0001D0310921C031092FB021092FA020E9439
:1008000027048FE893E00E94750485E693E00C943A
:100810007004CF93C62F0E94F7038C2FCF910C94B6
:1008200045047093F8026093F7020895E9EEF2E050
:100830001382128288EE93E0A0E0B0E08483958377
:10084000A683B7838AE191E0918380830895109213
:10085000AB0381E08093A9031092A80361E082E1D9
:100860000E94050961E083E10E940509E9EBF0E0DF
:1008700080818E7F808380818D7F808380E28093E2
:10088000B80085E48093BC000895880F8093BA0077
:10089000089520916003260F3327331F213231053D
:1008A000ECF42091AB03FC0190E080E0243069F08F
:1008B00082E00895A09160032191AC014E595C4FF4
:1008C000A40FB52FB11D2C930196861798F3809134
:1008D0006003680F6093600380E0089581E00895ED
:1008E0009093A5038093A40308959093A703809306
:1008F000A603089585ED8093BC008091BC0084FD23
:10090000FCCF1092AB03089585EC8093BC0010924D
:10091000AB0308951F920F920FB60F9211242F93DD
:100920003F934F935F936F937F938F939F93AF9377
:10093000BF93EF93FF938091B900887F803609F4CD
:100940004CC008F03FC0883209F4A8C018F58031C7
:1009500009F49CC0B8F4882309F4F9C0883009F47C
:1009600095C0FF91EF91BF91AF919F918F917F9132
:100970006F915F914F913F912F910F900FBE0F900C
:100980001F901895883109F489C0803251F78093FF
:100990003E0315C0803409F49EC048F48033B9F397
:1009A0008833F9F680933E030E948404DACF8035C1
:1009B00009F485C0883509F496C0883491F60E9400
:1009C0007A04CFCF883909F48CC038F5883729F0FC
:1009D00050F4883611F0803721F683E08093AB0322
:1009E00010923F0357C0883809F47BC0803919F052
:1009F000803809F0B6CF80913F03803208F071C093
:100A0000E0913F0381E08E0F80933F038091BB0014
:100A1000F0E0E05CFC4F80833DC0803B39F0E0F4C7
:100A2000803A09F479C0883A09F09BCF84E080933A
:100A3000AB031092610310926003E091A603F09162
:100A4000A70309958091600381110FC081E0809315
:100A500060031092620309C0803C09F476C0883CB0
:100A600009F473C0883B09F07CCFE091610381E019
:100A70008E0F80936103F0E0EE59FC4F80818093EC
:100A8000BB00909161038091600329C08091AA030B
:100A90008093BB0085EC8093BC0063CF909183036F
:100AA00080918203981758F5E091830381E08E0FBF
:100AB00080938303F0E0EC57FC4F8081E9CFE09115
:100AC000830381E08E0F809383038091BB00F0E06D
:100AD000EC57FC4F80839091830380918203981799
:100AE000C8F285E8D8CFE091830381E08E0F809330
:100AF00083038091BB00F0E0EC57FC4F8083809132
:100B0000A90381115CCF81E08093A80384EA8093DC
:100B1000BC001092AB0325CF0E94840480913F0358
:100B2000803230F4E0913F03F0E0E05CFC4F108253
:100B300060913F0370E0E091A403F091A50380E48D
:100B400093E0099510923F030CCF85ECE0CF109213
:100B50003E0335CF0F931F93CF93DF93EC01162FF6
:100B6000042F81E090E09983888386E391E09F835E
:100B70008E8380EF9AEBA4E0B0E088879987AA87FC
:100B8000BB8780E29EE4A0E0B0E08C879D87AE87C3
:100B9000BF87673120F08FEF9FEF998388830731FC
:100BA00020F08FEF9FEF9983888361E0812F0E946F
:100BB000C90860E0802F0E94C90860E0812F0E9470
:100BC0000509812F90E0FC01E158FF4FE491E88F87
:100BD000FC01EA56FF4FE491F0E0EE0FFF1FE355F2
:100BE000FF4F859194919A8F898F10E0F801E15819
:100BF000FF4FE491EB8FF801EA56FF4FE491F0E0EC
:100C0000EE0FFF1FE355FF4F859194919D8F8C8FC1
:100C10008FEF9FEFAFEFBFE08A839B83AC83BD83F1
:100C20000E94A607688B798B8A8B9B8BDF91CF9173
:100C30001F910F910895CF93DF93EC01F894E98D04
:100C4000FA8D9281888D809589238283EC8DFD8D2C
:100C500091818B8D809589238183EC8DFD8D92818F
:100C60008B8D809589238283EC8DFD8D81819B8D79
:100C7000892B8183EC8DFD8D92818B8D80958923CD
:100C800082838AE090E00E941008EC8DFD8D9181B6
:100C90008B8D809589238183EC8DFD8D92818B8D49
:100CA000809589238283E98DFA8D8281988D892BA5
:100CB00082837894EC8DFD8D3B8D488559856A85BE
:100CC0007B8520818C899D89AE89BF89232369F426
:100CD00084179507A607B70740F40196A11DB11D1B
:100CE0008C8B9D8BAE8BBF8BECCF481759076A0757
:100CF0007B0728F48EEF9FEFDF91CF910895F89452
:100D0000EC8DFD8D82819B8D892B8283EC8DFD8DF9
:100D100081819B8D892B8183EC8DFD8D82819B8DC3
:100D2000892B8283EC8DFD8D91818B8D809589231C
:100D30008183EC8DFD8D92818B8D809589238283BB
:100D4000E98DFA8D9281888D8095892382837894AC
:100D5000EC8DFD8D3B8D488559856A857B8520818D
:100D60008C899D89AE89BF89232349F4841795070F
:100D7000A607B70708F0BECF81E090E0BDCF84178B
:100D80009507A607B70708F0B5CF0196A11DB11DBD
:100D90008C8B9D8BAE8BBF8BE2CFCF92DF92EF928D
:100DA000FF921F93CF93DF93EC011C8A1D8A1E8A4A
:100DB0001F8A662309F473C08881998197FD73C0E7
:100DC000162FF12CCE010E941B0697FD70C0F394E4
:100DD0001F11F8CF0E94A607C888D988EA88FB8827
:100DE0006C197D098E099F09CC84DD84EE84FF8413
:100DF000C616D706E806F90678F5CA80DB80EC80CF
:100E0000FD80C701B6010E94A3092DEC3CEC4CEC1F
:100E10005DE30E94310A0E946D09AB01770F660BFA
:100E2000770B8C899D89AE89BF898C199D09AE0984
:100E3000BF0984179507A607B70770F48FEF9FEFD8
:100E4000AFEFBFE08A839B83AC83BD830E94A6077C
:100E5000688B798B8A8B9B8B8C899D89AE89BF89A6
:100E6000CA80DB80EC80FD808C159D05AE05BF053A
:100E700020F48A839B83AC83BD83CA80DB80EC80B3
:100E8000FD80BC01CD016C197D098E099F09DF91A0
:100E9000CF911F91FF90EF90DF90CF90089560E089
:100EA00070E0CB01F4CF6FEF7FEFCB01F0CF6EEFAF
:100EB0007FEF8FEF9FEFEBCF1F920F920FB60F9246
:100EC00011242F933F938F939F93AF93BF93809160
:100ED000B1039091B203A091B303B091B4033091E8
:100EE000B00326E0230F2D3768F129E8230F03967E
:100EF000A11DB11D2093B0038093B1039093B20361
:100F0000A093B303B093B4038091AC039091AD036D
:100F1000A091AE03B091AF030196A11DB11D8093C6
:100F2000AC039093AD03A093AE03B093AF03BF9116
:100F3000AF919F918F913F912F910F900FBE0F9086
:100F40001F9018950296A11DB11DD4CF2FB7F8940C
:100F50006091B1037091B2038091B3039091B40397
:100F60002FBF08953FB7F8948091AC039091AD03E3
:100F7000A091AE03B091AF0326B5A89B05C02F3F4B
:100F800019F00196A11DB11D3FBFBA2FA92F982FAF
:100F90008827BC01CD01620F711D811D911D43E0A9
:100FA000660F771F881F991F4A95D1F708958F9272
:100FB0009F92AF92BF92CF92DF92EF92FF926B011E
:100FC0007C010E94B2074B015C01C114D104E10411
:100FD000F104E9F00E946C090E94B20768197909CE
:100FE0008A099B09683E73408105910570F321E0F1
:100FF000C21AD108E108F10888EE880E83E0981E35
:10100000A11CB11CC114D104E104F10429F7FF9023
:10101000EF90DF90CF90BF90AF909F908F9008950A
:10102000000000008330910528F0880F991F059774
:101030000197F1F70895789484B5836084BD85B5F0
:10104000836085BDEEE6F0E0808181608083E1E829
:10105000F0E082E08083808181608083E0E8F0E0DE
:10106000808181608083E1EBF0E080818460808317
:10107000E0EBF0E080818160808386E880937A00F5
:101080001092C10008951F93CF93DF93182FEB01A7
:1010900061E00E94C908209739F460E0812FDF9158
:1010A000CF911F910C940509CF3FD10511F461E058
:1010B000F5CFE12FF0E0E859FF4FE491E43031F152
:1010C00040F4E230B1F0E330E1F0C038D1057CF714
:1010D000E4CFE83029F1E93059F1E530B1F78091FA
:1010E0008000806280938000D0938B00C0938A0040
:1010F00004C084B5806884BDC7BDDF91CF911F91C6
:10110000089584B5806284BDC8BDF7CF809180000A
:10111000806880938000D0938900C0938800EDCFD1
:101120008091B00080688093B000C093B300E5CF99
:101130008091B00080628093B000C093B400DDCF96
:10114000843081F028F48230E9F08330F9F008959A
:10115000883071F0893091F08530B9F48091800049
:101160008F7D03C0809180008F77809380000895E9
:101170008091B0008F778093B00008958091B00087
:101180008F7DF9CF84B58F7784BD089584B58F7D29
:10119000FBCFCF93DF9390E0FC01E158FF4F249108
:1011A0008A569F4FFC0184918823C9F090E0880FF4
:1011B000991FFC01EF53FF4FA591B491FC01E95435
:1011C000FF4FC591D49161110DC09FB7F8948C91D8
:1011D000209582238C938881282328839FBFDF91C9
:1011E000CF910895623051F49FB7F8943C91822FCB
:1011F000809583238C93E8812E2BEFCF8FB7F894C3
:10120000EC912E2B2C938FBFEACF1F93CF93DF93BC
:10121000282F30E0F901E859FF4F8491F901E15896
:10122000FF4FD491F901EA56FF4FC491CC23A9F0A6
:10123000162F81110E94A008EC2FF0E0EE0FFF1F87
:10124000E954FF4FA591B4918FB7F894EC91111127
:1012500008C0D095DE23DC938FBFDF91CF911F9123
:101260000895DE2BF8CFCF93DF93282F30E0F901DC
:10127000E859FF4F8491F901E158FF4FD491F901EA
:10128000EA56FF4FC491CC23A1F081110E94A0081F
:10129000EC2FF0E0EE0FFF1FE355FF4FA591B49147
:1012A000EC91ED2381E090E009F480E0DF91CF91B3
:1012B000089580E090E0FACF08950E941B080E94F4
:1012C0005C090E949200C0E0D0E00E94B502209725
:1012D000E1F30E940000F9CF08950E947409689418
:1012E000B1110C942B0A08950E94100A88F09F57A0
:1012F00098F0B92F9927B751B0F0E1F0660F771F3A
:10130000881F991F1AF0BA95C9F714C0B13091F02F
:101310000E942A0AB1E008950C942A0A672F782FB8
:101320008827B85F39F0B93FCCF3869577956795F4
:10133000B395D9F73EF490958095709561957F4F60
:101340008F4F9F4F0895E89409C097FB3EF4909506
:101350008095709561957F4F8F4F9F4F9923A9F08E
:10136000F92F96E9BB279395F6958795779567951D
:10137000B795F111F8CFFAF4BB0F11F460FF1BC061
:101380006F5F7F4F8F4F9F4F16C0882311F096E9F4
:1013900011C0772321F09EE8872F762F05C06623A2
:1013A00071F096E8862F70E060E02AF09A95660F5B
:1013B000771F881FDAF7880F9695879597F9089514
:1013C00097F99F6780E870E060E008959FEF80ECF8
:1013D000089500240A94161617061806090608959B
:1013E00000240A9412161306140605060895092E01
:1013F0000394000C11F4882352F0BB0F40F4BF2B70
:1014000011F460FF04C06F5F7F4F8F4F9F4F0895AF
:1014100057FD9058440F551F59F05F3F71F04795A5
:10142000880F97FB991F61F09F3F79F0879508958A
:10143000121613061406551FF2CF4695F1DF08C0A9
:10144000161617061806991FF1CF869571056105C6
:1014500008940895E894BB2766277727CB0197F96E
:1014600008950E94440A0C94F7090E94E90938F093
:101470000E94F00920F0952311F00C94E0090C94DF
:10148000E60911240C942B0A0E94080A70F3959F18
:10149000C1F3950F50E0551F629FF001729FBB276B
:1014A000F00DB11D639FAA27F00DB11DAA1F649F07
:1014B0006627B00DA11D661F829F2227B00DA11DBA
:1014C000621F739FB00DA11D621F839FA00D611D40
:1014D000221F749F3327A00D611D231F849F600D61
:1014E000211D822F762F6A2F11249F5750409AF08A
:1014F000F1F088234AF0EE0FFF1FBB1F661F771F16
:10150000881F91505040A9F79E3F510580F00C94E0
:10151000E0090C942B0A5F3FE4F3983ED4F38695E0
:1015200077956795B795F795E7959F5FC1F7FE2B80
:10153000880F911D9695879597F90895EE0FFF1FD7
:0C1540000590F491E02D0994F894FFCF81
:10154C0001010114150607080E010203040506012A
:10155C00020304050607000000009B03CA033803BE
:08156C0064033B034203550335
:00000001FF
